:1000000000308A0089280000FF00030E8301A10050
:100010007F08A0000A08A8008A01A00E0408A20018
:100020007708A3007808A4007908A5007A08A6003C
:100030007B08A700831383128C308400001C2228C5
:100040000C183B288C308400801C28288C183D28F4
:10005000220884002308F7002408F8002508F90086
:100060002608FA002708FB0028088A00210E8300D2
:10007000FF0E7F0E09008A113F288A1153282F1482
:100080000C108A1128280830BD02031C52283D306C
:1000900084000310800C00080319522850286400C3
:1000A000800B4F2800348316051183120515640058
:1000B0000930BC006D30BD004320BC0B5A282C0811
:1000C000BB00BB0803196A286400000000000000A0
:1000D000BB03612883160511831205118C108A1148
:1000E00028283A3084000008031988280230F800D4
:1000F000BF30F7006400F70B7A28F80B78289630A9
:10010000F700F70B8128000000006400800B7628C0
:10011000003484011F308305703083168F001F1256
:100120009F121B0880399B0007309C008312B80186
:1001300083161F129F121B0880399B001F13831206
:100140001F179F1783169F1383121F149412831671
:100150000611861406123130831294000030831683
:1001600094000108C73908388100B5308312900027
:100170007830F800063892008C3083169200723086
:100180008F000513831205138316851383128513BD
:1001900083160510831205108316851083128510AF
:1001A000B101B001B301B2018030AC00AE018316E1
:1001B0008C140C14C03083128B0483160611831226
:1001C00006110430B900FA30BA007120B90BE328E7
:1001D000A030AD000108801FF028B11FF828F228D8
:1001E000B11B0129B108031DF8283002031C0129A5
:1001F000831685108312851083160510831205144B
:1002000009298316051083120510831685108312A1
:1002100085100108801F0F29B31F17291129B31B4F
:100220002029B308031D17293202031C2029831635
:100230008513831285138316051383120517282946
:1002400083160513831205138316851383128513F2
:1002500064000130BA0071200230B900A9018B1B83
:10026000A9178B13F730BD004320A91B8B17B90BBF
:100270002E292A08B700B80A831606108312061022
:1002800013089301831614184729831242298312F5
:100290001308AA00AA098316061083120614003058
:1002A0002F180130003A031D6B290F08FA000E08C1
:1002B000F7000F087A02031D55297708B9007A085C
:1002C000BA003A08FA01FF3CB600B60CB60CB60C00
:1002D0001F30B6056D29B6012F10B501B4013408E1
:1002E000063C031C81292A08F7003408F80003198A
:1002F0007D290310F70CF80B79297718B50AB40A91
:100300006F293508033C03189629831605138312B9
:100310000513831685138312851383160510831224
:10032000051083168510831285108529AA1F982928
:10033000AA1DAF298030AC00FA012D08B0007A0860
:10034000B100FA012D08B2007A08B3000230AB0008
:100350008F018E012E0FAD29AE29AE0AEA282A1C84
:10036000CD2937082A020319B8293608583CAC00B1
:100370003808093C0318C129B8012C08573C031858
:10038000AC0AB101B001FA012D08B2007A08B3003D
:100390000130AB008F018E01EA282A1FEA293708B5
:1003A0002A020319D629A8303607AC003808093CC0
:1003B0000318DF29B8012C08A83C031CAC03B301C7
:1003C000B201FA012D08B0007A08B100AB018F012B
:1003D0008E01EA28AA1C0C2A37082A020319F329DD
:1003E0003608763CAC003808093C0318FC29B801F3
:1003F0002C08753C0318AC0A32302D02FA01B0000B
:100400007A08B100FA012D08B2007A08B300023070
:10041000AB008F018E01EA28AA1E2E2A37082A0275
:100420000319152A8A303607AC003808093C03182E
:100430001E2AB8012C088A3C031CAC0332302D0262
:10044000FA01B2007A08B300FA012D08B0007A0868
:10045000B1000230AB008F018E01EA282A1D532A19
:1004600037082A020319372A36087A3CAC003808C4
:10047000093C0318402A2C08793C0318AC0AB8013F
:10048000FA012D08B0007A08B100FA012D08B20077
:100490007A08B3000230AB008F018E012E0F512A73
:1004A000522AAE0AEA282A1E782A37082A02031995
:1004B0005C2A86303607AC003808093C0318652AE8
:1004C000B8012C08863C031CAC03FA012D08B200CD
:1004D0007A08B300FA012D08B0007A08B1000230A2
:1004E000AB008F018E012E0F762A772AAE0AEA28FA
:1004F0002B0B7B2A7E2AAB08031D982A2E08FA3C78
:100500000318952A8316051083120510831685108B
:10051000831285148316051383120513831685131E
:10052000831285176430BA007120AE01A030AD008F
:04053000EA28630052
:04400E00383FFC3FFC
:00000001FF
